:1000000081C000009AC0000098C0000096C00000A7
:1000100094C0000092C0000090C000008EC000009C
:100020008CC000008AC0000088C0000080C20000B0
:1000300084C0000082C0000080C0000093C00000A7
:100040007CC000007AC0000078C0000076C00000CC
:1000500074C0000072C0000070C000006EC00000DC
:100060006CC000006AC0000068C0000066C00000EC
:1000700064C000001201100102000008EB036F20B1
:1000800001000102000109023E00020100C0320924
:1000900004000001020201000524001001042402F2
:1000A000060524060001070582030800FF09040174
:1000B00000020A0000000705040210000107058382
:1000C00002100001040309041803500049004E0007
:1000D000470020004C00610062007300000026030E
:1000E000460072006900640067006500200043005C
:1000F0006F006E00740072006F006C006C00650091
:100100007200000011241FBECFEFD2E0DEBFCDBFD2
:1001100011E0A0E0B1E0EEECFEE002C005900D922F
:10012000A83DB107D9F712E0A8EDB1E001C01D92DA
:10013000A631B107E1F7EBD0C8C662CFE0E8F0E046
:10014000F0938900E093880088E0808384E08093C6
:10015000810082E080936F00089510920802089554
:10016000089508951F920F920FB60F9211248F9346
:100170001D992C9A809108028F3F61F080910802AE
:100180008E3120F4809108028F5F02C02C9A8FEF8D
:10019000809308028F910F900FBE0F901F901895BB
:1001A00080EC91E0ADC580EC91E061C584B7877FBC
:1001B00084BF2EE088E190E00FB6F894A895809374
:1001C00060000FBE2093600090E080E80FB6F894C6
:1001D00080936100909361000FBE9AC1CF93DF932B
:1001E000EC018DE191E0BE01F8D5009739F485B1BD
:1001F00090E2892785B982E291E04EC086E391E0E2
:10020000BE01EBD5009731F08DE391E0BE01E5D55D
:10021000009751F480E191E06AEF71E013D61092FB
:10022000D7011092D6013BC083E491E0BE01D5D541
:10023000009751F48AE491E06AEF71E003D685B14A
:1002400090E1892785B92BC081E691E0BE01C5D533
:10025000009739F486E691E06AEF71E0F3D52C9AC5
:100260001EC086E791E0BE01B8D5009741F48DE746
:1002700091E06AEF71E0E6D52C986FDF10C08FE84F
:1002800091E0BE01AAD5009751F41D9B03C08AE9F5
:1002900091E002C08CEA91E06AEF71E0D3D5DF9182
:1002A000CF910895CF93DF9328C0CE016AEF71E01C
:1002B0009DD5CD30D10599F48AE090E06AEF71E0E8
:1002C00095D58091D901E82FF0E0E652FE4F1082DB
:1002D0008F5F8093D9018AED91E080DF0CC080911F
:1002E000D901E82FF0E0E652FE4FC0838F5F809384
:1002F000D901803211F41092D90180EC91E0FCD345
:10030000EC01181619068CF2DF91CF910895CF9366
:10031000DF9381E184B915B849DF10DF80EC91E00B
:100320006AEF71E016D47894C0E9D1E00DC0A895C9
:1003300084EC99E0FE013197F1F70197D9F7B2DF2C
:1003400080EC91E050D4C4D38091D6019091D70134
:10035000892B69F78091E00081608093E0002CE0B8
:1003600088E190E00FB6F894A895809360000FBEE6
:1003700020936000FFCFDA01923049F0933061F0B2
:100380009130F9F4E4E7F0E022E130E01EC0E6E865
:10039000F0E02EE330E019C0813049F0813018F0F0
:1003A000823079F408C0E4ECF0E0849107C0E8EC16
:1003B000F0E0849103C0EEEDF0E08491282F30E06E
:1003C00004C0E0E0F0E020E030E0ED93FC93C901F0
:1003D00008958093E9008091EB0081608093EB00A9
:1003E0001092ED006093EC004093ED008091EE00E0
:1003F000881F8827881F089580910E0288239CF407
:1004000004C080910D028823B9F08091E80082FF3A
:10041000F8CF8091E8008B778093E8000895809171
:100420000D02882349F08091E80080FFF8CF809189
:10043000E8008E778093E80008954091E4005091A1
:10044000E50024E68091EC0080FF05C08091E80083
:1004500080FF05C022C08091E80082FD1EC080910F
:100460000D02882311F482E00895853011F483E0B1
:1004700008958091EB0085FF02C081E0089580918E
:10048000E4009091E50084179507E1F2222311F42E
:1004900084E008952150AC01D5CF80E0089541D08B
:1004A00043D08091D800982F9F779093D800806890
:1004B0008093D80084E089BD89B5826089BD09B484
:1004C00000FEFDCF8091D8008F7D8093D8001092E0
:1004D0000D0210920B0210920A021092090280E0A3
:1004E00060E042E076DF8091E1008E7F8093E10062
:1004F0008091E20081608093E2008091E200886058
:100500008093E2008091E0008E7F8093E000089568
:10051000E3E6F0E080818E7F808381E080930C02AF
:10052000BECF1092E20008951092E10008951F924C
:100530000F920FB60F9211242F933F934F935F9317
:100540006F937F938F939F93AF93BF93EF93FF939B
:100550008091E10080FF1CC08091E20080FF18C004
:100560008091E1008E7F8093E1008091E2008E7F98
:100570008093E2008091E20080618093E2008091AC
:10058000D80080628093D80019BC10920D02E9DD7A
:100590008091E10084FF2EC08091E20084FF2AC098
:1005A00084E089BD89B5826089BD09B400FEFDCFB4
:1005B0008091D8008F7D8093D8008091E1008F7E5C
:1005C0008093E1008091E2008F7E8093E200809131
:1005D000E20081608093E20080910B02882331F475
:1005E0008091E30087FD02C081E001C084E0809338
:1005F0000D02B6DD8091E10083FF22C08091E20010
:1006000083FF1EC08091E100877F8093E10082E03C
:1006100080930D0210920B028091E1008E7F8093F7
:10062000E1008091E2008E7F8093E2008091E20001
:1006300080618093E20080E060E042E0CADE4BD15E
:100640008091E10082FF0AC08091E20082FF06C033
:100650008091E1008B7F8093E1003DD1FF91EF918C
:10066000BF91AF919F918F917F916F915F914F91CA
:100670003F912F910F900FBE0F901F9018950F93E1
:100680001F93DF93CF9300D0CDB7DEB7EEE0F2E05B
:100690008091F100819382E0E631F807C9F780DDAF
:1006A0008091E80083FF02C180910E0230910F0219
:1006B000353009F487C0363040F43130C9F131307B
:1006C00070F0333009F0F2C033C0383009F4C0C0E4
:1006D000393009F4CFC0363009F0E8C099C080380D
:1006E00021F0823809F0E2C008C09091090280919F
:1006F0000A02882399F0926011C0809112028770DB
:100700008093E9008091EB0090E025E09695879535
:100710002A95E1F7982F91701092E9008091E800F6
:10072000877F8093E8009093F1001092F1009BC0C6
:10073000882319F0823009F0B9C090E08F71907071
:10074000009721F0029709F0B1C00CC0809110020F
:10075000813009F0ABC010920A02333069F5809302
:100760000A022AC080911002882331F520911202DA
:10077000277009F49BC02093E9008091EB0080FF73
:100780001BC0333021F48091EB00806213C0809154
:10079000EB0080618093EB0081E090E002C0880F65
:1007A000991F2A95E2F78093EA001092EA0080915F
:1007B000EB0088608093EB001092E9008091E800E4
:1007C000877F54C0882309F071C0109110021F77F1
:1007D0000FB7F8948091E800877F8093E8000CDEE3
:1007E0008091E80080FFFCCF112311F482E001C06A
:1007F00083E080930D028091E3008078182B1093A2
:10080000E3008091E30080688093E3000FBF4EC057
:100810008058823008F04AC08091100290911102F5
:1008200060911202AE014F5F5F4FA5DDBC010097E2
:1008300009F43CC08091E800877F8093E8008981BB
:100840009A81A8D08091E8008B778093E8002EC031
:10085000803861F58091E800877F8093E80080917F
:100860000B028093F1008091E8008E778093E8007E
:10087000C3DD1CC08823D1F4909110029230B0F4F3
:100880008091E800877F8093E80090930B02B4DDAD
:1008900080910B02882331F48091E30087FD02C030
:1008A00081E001C084E080930D027DDC8091E8004E
:1008B00083FF0AC08091EB0080628093EB008091FF
:1008C000E800877F8093E8000F900F90CF91DF9131
:1008D0001F910F91089508959C0140911402509129
:1008E00015024617570718F4F90190E03DC061154D
:1008F000710511F0AB01F8CF8091E8008E778093FD
:10090000E80040E050E0F0CF80910D028823F1F143
:100910008530F1F18091E80083FF02C081E0089505
:100920008091E80082FD2CC08091E80080FF1CC00F
:100930008091F200282F30E007C081918093F10070
:10094000415050402F5F3F4F4115510519F028305D
:10095000310598F390E02830310509F491E0809159
:10096000E8008E778093E8004115510569F69923D8
:1009700059F606C080910D02882341F0853041F080
:100980008091E80082FFF6CF80E0089582E008952C
:1009900083E008959C01409114025091150246177E
:1009A000570710F460E03FC06115710511F0AB010D
:1009B000F9CF8091E8008E778093E80040E050E026
:1009C000F1CF80910D02882309F43FC0853009F4EE
:1009D0003EC08091E80083FF02C081E008958091CD
:1009E000E80082FD2CC08091E80080FF1CC080914F
:1009F000F20090E009C0F9012F5F3F4FE491E093CE
:100A0000F1004150504001964115510519F08830D0
:100A1000910588F360E0089709F461E08091E800AF
:100A20008E778093E8004115510559F6662349F603
:100A300006C080910D02882341F0853041F08091FD
:100A4000E80082FFF6CF80E0089582E0089583E019
:100A500008959C016115710529F48091E8008B7758
:100A60008093E800F90120C080910D02882361F194
:100A7000853061F18091E80083FF02C081E0089534
:100A80008091E80082FFF0CF06C08091F100819351
:100A90006150704021F08091F2008823B1F780917D
:100AA000E8008B778093E80061157105E9F606C0D0
:100AB00080910D02882341F0853041F08091E8005B
:100AC00080FFF6CF80E0089582E0089583E00895E6
:100AD0001F9380910D02882361F01091E90010921C
:100AE000E9008091E80083FF01C0C9DD1770109311
:100AF000E9001F9108950895FC0180910D02843052
:100B000021F587859089A189B2890097A105B10552
:100B1000E1F085818093E9008091E80082FF15C0B3
:100B20008091F200882319F42FEF3FEF04C08091E9
:100B3000F100282F30E08091F200882341F4809169
:100B4000E8008B778093E80002C02FEF3FEFC901E8
:100B50000895FB012EE0DB011D922A95E9F723E0C1
:100B6000238328E236E0318720872CEB35E033877A
:100B70002287958784870895FC0184859585BCDF4D
:100B80009C0197FF02C02EEF3FEFC9010895FC01C1
:100B900080910D02843011F587859089A189B289F1
:100BA0000097A105B105D1F081818093E900809182
:100BB000F2008823A9F09091E8008091E8008E77F8
:100BC0008093E80095FD0CC038DC982F882349F409
:100BD0008091E8008E778093E80003C092E001C026
:100BE00090E0892F0895FC0180910D02843051F42A
:100BF00087859089A189B2890097A105B10511F077
:100C0000CF01C5CF08951F93FC01162F80910D02CF
:100C10008430D9F487859089A189B2890097A1058C
:100C2000B10599F081818093E9008091E80085FD0C
:100C300008C08091E8008E778093E800FEDB88236F
:100C400029F41093F10080E001C082E01F91089523
:100C5000282FFB0184859585622FD5DF882319F421
:100C600020E030E002C02FEF3FEFC90108951F934D
:100C7000CF93DF93EC010D96FC0189E0DF011D921B
:100C80008A95E9F711E08981181729F4EA81FB8137
:100C90008C8162E010C08D81181731F4EE81FF81E4
:100CA000888562E030E008C08985181709F5EA8573
:100CB000FB858C8563E031E0882311F440E001C0BE
:100CC00044E020E088E090E003C02F5F880F991F88
:100CD0008E179F07D0F36295660F660F607C632BBB
:100CE00042602295207F422B812F73DB882321F0E5
:100CF0001F5F153041F681E0DF91CF911F9108957C
:100D0000CF93DF93EC018091E80083FF63C088817B
:100D100090E020911202309113022817390709F050
:100D200059C080910F02813261F0823220F480320A
:100D300009F050C01BC0823279F1833209F04AC0F9
:100D40003BC080910E02813A09F044C08091E800D6
:100D5000877F8093E800CE010F9667E070E0BCDDEE
:100D60008091E8008B778093E80034C080910E0278
:100D7000813281F58091E800877F8093E800CE0181
:100D80000F9667E070E065DE8091E8008E778093D3
:100D9000E800CE01B0DE1EC080910E028132D1F497
:100DA0008091E800877F8093E80026DB8091100225
:100DB0008D87CE01A0DE0EC080910E02813251F4EB
:100DC0008091E800877F8093E80016DBCE01609178
:100DD000100291DEDF91CF910895FB01DC018D912E
:100DE000019080190110D9F3990B08950F931F9367
:100DF000CF93DF938C01EB018B8181FF1BC082FFBE
:100E00000DC02E813F818C819D812817390764F4A4
:100E1000E881F9810193F983E88306C0E885F985C3
:100E2000802F0995892B31F48E819F8101969F83B4
:100E30008E8302C00FEF1FEFC801DF91CF911F918A
:100E40000F910895EF92FF920F931F93CF93DF932B
:100E50007C018B01DB0113968C9181FD03C0CFEFE8
:100E6000DFEF13C0C0E0D0E00BC0D8011896ED91C1
:100E7000FC911997B8010995892B11F0CFEFDFEF9D
:100E8000F70181917F01882381F7CE01CDB7DEB7CD
:100E9000E6E00CC02A88398848885F846E847D84A7
:100EA0008C849B84AA84B984C884DF80EE80FD8012
:100EB0000C811B81AA81B981CE0FD11D0FB6F89488
:0E0EC000DEBF0FBECDBFED010895F894FFCF49
:100ECE0048656C6C6F2C20576F726C64210D0A0094
:100EDE005265626F6F74696E67210D0A00636F6CE5
:100EEE0061006D6D6D21204C454420746F67676500
:100EFE006C65640D0A007265626F6F7400726573C3
:100F0E00657400746F67676C6500546F67676C6912
:100F1E006E67204D61676E6574204C6F636B0D0AB2
:100F2E00006C6F636B007374617475733A206C6F31
:100F3E00636B65640A00756E6C6F636B007374612E
:100F4E007475733A20756E6C6F636B65640A00641A
:100F5E006F6F7273746174757300646F6F727374F4
:100F6E00617475733A206F70656E0A00646F6F72EC
:100F7E007374617475733A20636C6F7365640A00E1
:100F8E000003100000041000000208000000000022
:080F9E0000000000000001004A
:00000001FF
